:020000020000FC
:1000000024C937C20000000023C000004FC1000017
:10001000000052C1000000000000000002030406BE
:10002000080C101820304060800002030406080C01
:10003000101820304080FF000406080C10182030F3
:10004000406080A0C00005050D050D0603030302F6
:100050004FB662FD20C070FF1CC165FDFCC057FE9D
:1000600001C00994C0919700C395C0939700C5E063
:10007000C519B8F3D0919700CD1B98F3C8E7089441
:1000800083FDC795C4BDC52DCC2321F4C0E083FDFD
:10009000C0E8C4BD09C171FF03C0C098C198C2982F
:1000A000C52D089483FDC795C4BDC09399006B7F8F
:1000B000C52DCF3F09F443C0C0919800C395C093AC
:1000C000980070FF37C082FD05C0C098C198C298E3
:1000D0004FBE18957860C091A000CC2391F0C091DC
:1000E0009800CA95D091A000CD1B58F0777FC091A1
:1000F0009800D0919F00CD1B08F41CC0209298005E
:1001000019C0C098C198C298C5E0CA95F1F7C091CE
:100110007500CA95C2FD09C0C1FD05C095FF959A3D
:1001200095FD939A0EC0949A0CC095FF939A95FDF5
:10013000959A07C0C098C198C2984FBE1895209252
:1001400099004FBE1895A5C0552021F095FFC09A83
:1001500095FDC29AC1989DC0552009F0C19A95FF9E
:10016000C29895FDC09895C0552021F095FFC29A80
:1001700095FDC09A95FFC09895FDC2988AC095FFDD
:10018000939895FD959895FF959895FD9398C5E062
:10019000CA95F1F7552021F095FFC09A95FDC29AB6
:1001A000C19877C095FF939895FD95989498C5E070
:1001B000CA95F1F7552021F095FFC09A95FDC29A96
:1001C000C19867C0949895FF939895FD9598C5E060
:1001D000CA95F1F7552009F0C19A95FFC29895FD8F
:1001E000C09857C0949895FF959895FD9398C5E051
:1001F000CA95F1F7552009F0C19A95FFC29895FD6F
:10020000C09847C095FF959895FD93989498C5E040
:10021000CA95F1F7552021F095FFC29A95FDC09A35
:1002200095FFC09895FDC29834C095FF959895FDAF
:10023000939895FF939895FD9598C5E0CA95F1F729
:10024000552021F095FFC29A95FDC09A95FFC09860
:1002500095FDC2981EC082FF1CC0C0917500C2FDF2
:100260000BC0C1FD11C095FF939895FD959895FF22
:10027000959895FD93980DC0C1FDF5CF95FF939886
:1002800095FD9598949805C0949895FF959895FD3F
:100290009398C52DC095089483FDC795C4BDC093A0
:1002A00099002092970064604FBE18954FB6C0E148
:1002B000C8BF6E7F4FBE18953FB68F7EABB7A07498
:1002C000A2118061A0E0ABBFA9B7AE7FA9BF7894AF
:1002D000A0916600AA2349F0A92FAF7151F1A09116
:1002E0006600AA95A093660024C040E050E0A0B349
:1002F00096FDA095A2FD4FEF96FFA3E096FDA2E02C
:10030000A5BFAA27A064AABF8D7FA0B396FDA09524
:10031000A2FD5FEF451749F7A8E161FDA0936600D4
:10032000A92FAF7119F0A8E1A093660040938D004A
:100330008160A0916700AA2331F0A0916700AA957F
:10034000A093670007C0A92FAF7121F08061AA2791
:10035000A064AABF80FF48C0A0918D004A2F8E7F65
:10036000A92FAF71C1F0403F08F040EFA42FA29534
:10037000AF704A0F5091B000533069F0A695A69522
:1003800050FD01C0A69552FD03C0A41B4A2F03C017
:100390004A0F08F44FEFA09196004A1708F44A2F2D
:1003A0004093610071FF08C0A091610050919200DC
:1003B000A51710F050936100A09161004091630077
:1003C000A41B70F04091CF00A40B50F0A0916300EB
:1003D000A40FA093630040F4AFEFA093630004C0A8
:1003E000A0916100A093630040916300A0919200EE
:1003F0004A1708F04A2F542EA52DA03408F0686043
:10040000A0916000A395A093600051F0F894A9B763
:10041000A160A9BF84FF02C0A0E4ABBF3FBE189596
:1004200041E050916600552331F0A92FAF7119F4C6
:100430005A9550936600A0918D00A13018F020923B
:1004400090000DC02092910020929A00A0919000FF
:10045000AF5FA093900018F0AFEFA0939000F894D6
:10046000A9B7A160A9BF84FF02C0A0E4ABBF3FBE93
:1004700018953FB64CB55DB58F7EABB7A074A21191
:100480008061A0E0ABBFA9B7AE7FA9BF789481FD22
:1004900026C096FFA2E096FDA3E0A5BF8260A0B3B0
:1004A00096FDA095A2FF05C040936400509365009F
:1004B00033C196FFA3E096FDA2E0A5BFAA27A064E2
:1004C000AABF8D7FA92FAF7109F417C140E0A0B377
:1004D00096FDA095A2FD11C140938D0004C196FF29
:1004E000A3E096FDA2E0A5BF8D7F61FF6BC096FFE4
:1004F000A2E096FDA3E0A5BFAA27A064AABF8260E0
:100500004093880050938900A09086004A19B090CB
:1005100087005B09BB24A2E0EA2EA22C483CA0E0A5
:100520005A0730F4A0E1BA2EE22CAAE0AA2E27C086
:100530004836A1E05A0730F4A8E0BA2EE22CAFE02A
:10054000AA2E1DC0403DA2E05A0730F4A4E0BA2E06
:10055000E22CAEE1AA2E13C0403AA5E05A0730F4CF
:10056000A2E0BA2EE22CACE3AA2E09C04839A8E0DA
:100570005A0728F4A1E0BA2EE22CA8E7AA2EC42E2E
:10058000A0918A00CA1AD52EA0918B00DA0ADD202C
:100590002AF4AFEFC094D094CA1ADA0A20928C00E1
:1005A000CA14DE0418F4A1E0A0938C0040938A00E2
:1005B00050938B00409188005091890040938600B1
:1005C00050938700A09164004A1BA09165005A0BCC
:1005D00094FD7CC093FD7AC092FD76C056954795F8
:1005E00091FD72C05695479590FD6EC0D52EC42ED4
:1005F000D694C79461FD0CC0AC2DAC51AD2DA2407A
:1006000008F07BC0DD2021F4AC2DA85C08F475C097
:10061000A0E0EA2E97FD08C0E090C200A091B400CF
:10062000A33011F4E090CA00AAEFEA0EF22CF21CFB
:10063000CE18DF084FB74170A091B400A330A9F4E1
:10064000442329F095FD11C0F894906204C095FFF1
:100650000CC0F8949F7DC098C198C29893989498C4
:10066000959871FD01C060687894442369F0A09169
:10067000B400A33031F4AFEFC094D094CA1ADA0AB0
:1006800003C040E050E022C0A091B400A33049F480
:10069000CC0CDD1CA5E0CA1AD20818F4A0E0CA2EC2
:1006A000D22CAFEFCA16D20418F04FEF50E00EC0B4
:1006B000F090A700CF9C412D000C441F50E008F0A3
:1006C00012C04FEF50E00FC05695479594FF07C0FA
:1006D000552309F04FEFA42FA6954A0F521D4F3F07
:1006E000520508F04FEF40938D00816061FF05C017
:1006F000AFE1A095A923AB299A2FA8E1A0936600AA
:10070000A92FAF7119F4AAE0A093660061FD04C09F
:10071000A92FAF7109F08F7EA6E0A0936700A92FE3
:10072000AF7119F4AAE0A0936700F894A9B7A1608B
:10073000A9BF84FF02C0A0E4ABBF3FBE189511E083
:100740000AC013E008C01AE006C01EE104C014E6A7
:1007500002C018EC00C005E1BB27BA95F1F70A9575
:10076000D9F71A95C1F708952AE338E709C020E3BD
:100770003CE806C02AE234EB03C025E238EC00C0B6
:10078000652CB1E05B2E12E095FD9F7D95FF906298
:10079000BB279498BA95F1F7552009F0C19ABA95FC
:1007A000F1F7C198BA95F1F7949ABA95F1F75520F7
:1007B00021F095FFC09A95FDC29AB091A800BA9514
:1007C000F1F795FFC09895FDC298B7E8BA95F1F793
:1007D0001A95D1F6022FB22FBA95F1F70A95D9F7EB
:1007E0003A9571F69498562C0895221B39E0001F13
:1007F0003A9509F40895221F211B18F4210F8894BB
:10080000F6CF0894F4CF622C722CB0E08894B395A4
:10081000221F331FE0F7379527958894912E802E5D
:10082000020B130B10F4192D082D10F4889401C03D
:100830000894661C771CBA9571F7172D062D08953C
:10084000322D11232AF43A9500951095031B130BB2
:10085000F894029F712C002D129F912C802C78947B
:10086000780C172D921C292DB4E06B2E2695179528
:1008700007956A94D9F7332321F000951095031B4F
:10088000130B0895089566FF21C01091740016950A
:10089000009173000795B0917700B01B0B2FB091BA
:1008A0007800B10B1B2F28F40038BFEF1B0740F076
:1008B00009C00F37120508F405C00FE710E002C0A9
:1008C00000E81FEF00937C0010937D00089566FF01
:1008D00039C000917C00B09179000B0F10917D0020
:1008E000B0917A001B1F20E030917D0033230AF481
:1008F0002A95B0917B002B1F1AF4203F40F00AC0CC
:100900002F3008F407C00FEF1FEF2FE003C000E007
:1009100010E020EF30916300B09192003B1718F483
:10092000332331F009C0B0917D00BB235AF004C0DD
:10093000B0917D00BB2332F40093790010937A00CC
:1009400020937B00089566FF2FC02091CD00009179
:100950007C00000F10917D00111F72DF11232AF41B
:100960000038BFEF1B0740F009C00F37120508F42D
:1009700005C00FE710E002C000E81FEF002352F0AF
:10098000B0916200B01B0B2F18F0013008F00AC0C4
:1009900001E008C000950F5FB09162000B0F08F0F6
:1009A00001C00FEF00937E00089566FF2DC02091D7
:1009B000CE0000917A0010917B0042DF11232AF4CF
:1009C0000130BFEF1B0740F009C00F3F120508F4CC
:1009D00005C00FEF10E002C001E01FEF112352F03D
:1009E000B0917E00B01B0B2F18F0013008F00AC048
:1009F00000E008C000950F5FB0917E000B0F08F07B
:100A000001C00FEF0093630008950FEF677FB72FCA
:100A1000B670E9F46860B0917400B83008F0677F90
:100A2000B0917400A1F00FEF10917400DEDEF89425
:100A3000B09170000B9F112D002D7894112309F0B7
:100A40000FEFB09195000B1710F4009195000093F3
:100A5000940008956FC0DDD274FFB0E074FDB1E082
:100A6000B068B064B7B9B6B1B068B064B6B967DEA3
:100A700074FFB0E074FDB1E0B068B064B7B9B6B16E
:100A8000B068B064B6B9B6B1B6FDFDCF04B115B16A
:100A9000B6B1BF77B6B902D32DE62093A30030E0FC
:100AA0003093A400732E7694622E6694620E731EA9
:100AB000262D372D0217130778F08090A300BDE68E
:100AC000B80DB093A3008090A400B0E0B81DB0931F
:100AD000A400260D371DEECF8090A3009090A400B7
:100AE0001091A40016950091A300079516950795FF
:100AF000B091A300B00FB093A100B091A400B11FBA
:100B0000B093A20023E0169507952A95E1F720916E
:100B1000AF002A9529F42092A3002092A4000AC0D5
:100B20002A9521F0800E911E2A95E1F78092A3006C
:100B30009092A40008952091AF00B6B1B6FDFBCF0E
:100B400004B115B1B6B1BF77B6B9B091A500B395F0
:100B5000B093A500B83060F12092A500B091CC0010
:100B6000BB2321F1112329F0B091A600BF3F61F012
:100B700009C0B091A6000B1739F020F4BB2321F077
:100B8000BA9502C0B395E1F300919200B093A6002C
:100B9000BA3F50F400ECB93F38F400E8B83F20F415
:100BA00000E4B73F08F400E0009392007F7E0895D0
:100BB000B0919200B39511F0B0939200B091A5005E
:100BC000B73009F47061089502E3F894B091D00051
:100BD0000B9F012D000C001F7894B09192000B1711
:100BE00010F0009192000093610000936300502E7A
:100BF00000939500089520927300B8E0B0937400BC
:100C000008952091800030918100F8940CB51DB5B5
:100C1000200F311F3BBD2ABD6160B0E1B8BF7894A1
:100C20002091710030917200009371001093720056
:100C3000021B130B2091730030917400622E732EEF
:100C4000B4E08B2EB2E09B2EB0917400B43010F063
:100C50008A949A94B83010F08A949A94769467940F
:100C60008A94E1F726193709992021F016950795FE
:100C70009A94E1F7200F311F209373003093740092
:100C800008F00895BFEFB0937300B0937400089517
:100C90002091820030918300F8940CB51DB5020FAD
:100CA000131F1BBD0ABD6160B0E1B8BF7894089501
:100CB00060FDFECFEDDF0895B091BE0000916E00A3
:100CC000023808F0B395003A08F0B395B63008F052
:100CD000B5E09B2EBCE08B2EB0917400B33030F4A5
:100CE0008394839482FF02C083948394B23030F45F
:100CF0008394839482FF02C08394839471FF03C022
:100D0000B3E09B2E822C109174000091730024E0BC
:100D1000169507952A95E1F70819120928F0B02FC2
:100D2000B250B12FB20910F402E010E0312F202FA1
:100D3000712E602E76946794B92DB330E9F0B0FD32
:100D400005C0060D171D262D372D06C0000F111FDB
:100D50000250120922E030E0B92DB33068F0209340
:100D6000840030938500009380001093810060928E
:100D70008200709283000895009384001093850090
:100D800020938000309381006092820070928300F3
:100D9000089560FDFECF20918200220F30918300E4
:100DA000331FB72FB67021F020917300309174007B
:100DB000F8940CB51DB5020F131F1BBD0ABD616071
:100DC000B0E1B8BF7894089560612092760020E089
:100DD00004C060612092760020E2B72FB67009F05F
:100DE0006F7E789460FD05C0B0917600BB2309F05A
:100DF000089501E063FF0AC0B0917400B33008F0B9
:100E000002E0B0917400B63008F003E071FF01C059
:100E100006E060FD06C0B0917600BB2311F0789427
:100E200008951AE083FF1AE0789400000000F89417
:100E300062FD03C014E183FF14E171FF01C018E7F4
:100E4000B4B530919900B31BB10B18F3B091760093
:100E5000B395B0937600B5E03B2F6B2E722CB8B1F2
:100E6000B072B21709F073943A95C9F77394761477
:100E700088F464FFB2CF6F7E3CB56DB470907300A0
:100E800080907400370D681C6BBC3ABD6160B0E1A6
:100E9000B8BFA3CF64FDA1CF0A9509F0BACF78946B
:100EA000089571FF0AC0B0916D00B395B0936D00C5
:100EB00060FD0CC020926D0009C060FD07C064FD9C
:100EC00005C067FD03C0BF91BF9182C40895209102
:100ED000840030918500F8940CB51DB5020F131FE6
:100EE0001BBD0ABD6160B0E1B8BF78940895EFDF23
:100EF00000E063FF03C064FF01C001E0F8941091BB
:100F00006E00B7E01B9F212D102D7894200F2695A1
:100F10001795269517952695179510936E001837F7
:100F200018F4B8E7B0936E0000916E00B0916F00B6
:100F30000B1720F06062C098C198C29860FDFECF88
:100F40000895F89493989498959882FF07C0E2E0EA
:100F5000F1E073FF03C0B5E0BA95F1F795FF939AFE
:100F600095FD959AB2E0B093750089C0F89495FF0D
:100F7000C29895FDC09882FF0DC0E2EFF0E073FFCC
:100F80000BC0949895FF959895FD9398B5E0BA9508
:100F9000F1F702C0ECEAF0E062FF03C0552009F06F
:100FA000C19AB3E0B09375006AC0F894939894988E
:100FB000959882FF07C0E2EEF0E073FF03C0B5E052
:100FC000BA95F1F795FF959A95FD939AB4E0B09391
:100FD000750055C0F894C19882FF0DC0E2EDF0E0B5
:100FE00073FF0BC095FF939895FD95989498B5E085
:100FF000BA95F1F702C0E4EAF0E062FF06C05520BE
:1010000021F095FFC09A95FDC29AB5E0B0937500A6
:1010100036C0F89493989498959882FF07C0EFEBA8
:10102000F0E073FF03C0B5E0BA95F1F7949AB6E02B
:10103000B093750024C0F89495FFC09895FDC298B0
:1010400082FF10C0E5E1F1E073FF0EC095FF9398B9
:1010500095FD959895FF959895FD9398B5E0BA956F
:10106000F1F702C0E4EBF0E062FF06C0552021F08A
:1010700095FFC29A95FDC09AB1E0B093750067FFE5
:101080000AC00CD0B5E0BA95F1F7B5E0BA95F1F722
:10109000939A949A959A6F7D7894089523EA30E014
:1010A000F901C098C198C2989398949895986B7FCD
:1010B0000895ACEAB0E00FEF0D930D930D930D93EF
:1010C00003E00D9304E00D9309E00D9303E00D930D
:1010D00001E00D9301E00D93A8EBB0E001E00D936A
:1010E0000FEF0D930D930FEF0D930D930D9303E001
:1010F0000D9306E00D930FEF0D930D9305E20D9305
:1011000000ED0D930AEF0D930AEF0D9304E00D939C
:101110000DE00D9301E00D9300E00D930AE70D93B0
:101120000FEF0D9301E00D9308952091BF0009E0AA
:1011300011E0223011F405E011E0233011F405E054
:1011400012E0243011F405E013E0253011F409E039
:1011500017E0263011F400E010E000939F00109398
:10116000A0002091B3008B7F233009F48460777F47
:10117000233009F47860B091B400B33019F09F7D4A
:10118000B1FD90629F7BB091B500B1FD9064B22F2C
:10119000B23011F0886001C0877F0895ECE1F0E083
:1011A0000091AC000A95E00FF21DB491B093CD0010
:1011B0000091AD000A95E00FF21DB491B093CE00FE
:1011C0006DDF0895EAE2F0E00091C7000A95E00FB4
:1011D000F21DB491B093CF0061DF0895E8E3F0E031
:1011E0000091B2000A95E00FF21DB491B093D000C7
:1011F00055DF08950895B091C8000FEF1CE0B2309C
:1012000011F400EA1AE0B33011F402E815E000939B
:101210006F0010937000089508952091C2003091DE
:10122000C30097FF02C020E03FEFB32FB21B6B2E2D
:10123000B25810F4B2E86B2E00E00395609EB12D19
:10124000B058D8F30093A7000895F894E3E0F0E0D5
:10125000B9E0B7BFB491B078C1F3F894A895B1B52F
:10126000B861B1BDB0E0B1BDB4E0BEBFBFE5BDBFC8
:1012700015DFB0E0B8BBB7E1B7BBB0E0B5BBB0E0DD
:10128000B4BBB0E0B2BBB8E3B1BB2224A0E0B0E095
:101290002D92AA31E9F7A0E6B0E00FEF2D920A9562
:1012A000E9F707DFB5D241DF79DF8CDF97DFA2DF17
:1012B000A2DFB2DFB2DF0091C4000093A800EEDE2F
:1012C000B2E0B3BFB2E0BEBDB2E0B5BDF89441DA62
:1012D0004BDA3BDA4CDA39DA4DDA37DA24D339DA59
:1012E00038DA35DAB1E5B8BFB9BFB0B7B860B0BF6A
:1012F000B6B1B460B6B923DA7894ACDBB0E4BBBF66
:10130000BB27B064BABF8D7F24DAB1E0B093690027
:10131000626025E0B0918C00BB2309F425E011DA6E
:10132000B0918D00B230A8F3B92FBF7100918F003A
:1013300000938E00B0938F00B01759F72A9551F79C
:101340006D7F96FFB3E096FDB2E0B5BFBB27B064FA
:10135000BABF8D7FFCD9F5D902E0B92FBF7109F46E
:1013600000E0B0918D00B017B0F3F894FDD9FCD92E
:10137000FBD97894EED920927F00B091B400B330BD
:1013800009F472C0DED9B091B800B13008F46CC075
:10139000B0916900B13008F467C0B92FBF71C1F0D6
:1013A000B0918D00BF3F08F45FC0F894E6D97894FF
:1013B000CED9B0918D00B130C0F7F894D5D9C3D94A
:1013C000D3D97894C4D9B0918D00BF3FB0F3DDC2BA
:1013D000B8E09B2E9068F89420DF7894B8D9F89400
:1013E0009F771BDF80908D00B0918D00BF37789480
:1013F00008F442C0A4D9F894C0D978949A9451F7CB
:10140000B82DB550B093C300A4D9F8942ED290D281
:101410007894BAE09B2E9068F894FFDE789497D980
:10142000F8949F77FADE80908D00B0918D00BF37E1
:10143000789478F784D9F89497D985D995D9789400
:101440009A9449F7B82DBB5FB093C20082D9F89443
:101450000CD27DD278947BD9F894DFDE7894B09169
:101460008D00BF3FC0F391C200918D00B0917F000D
:101470000B1710F000937F006AD901E0B091B4001F
:10148000B35009F405E0B0918D00B01708F075CFA6
:10149000F89473D972D971D978945BD92092690084
:1014A00020926A0020926B00B0916A00B395B093CD
:1014B0006A00BF3F69F5B0916B00B395B0936B00C4
:1014C000B091C60009E1BA9559F002E3BA9541F02E
:1014D0000DE7BA9529F00AEFBA9511F020926B004A
:1014E000B0916B00B017A0F0B0916B00BA95B093BB
:1014F0006B00B4EBB0936A00B091C500B093A80044
:10150000F8943BD97894B091C400B093A8001FD947
:101510001AD9B0916600BB2321F4B92FBF7109F429
:10152000F7CEB0918D00B63008F4BECFB091B400C4
:10153000B35009F00CD9B0916600BB2309F4E8CE92
:10154000F894ACDD2092610020926200209263004A
:10155000522C7894B091B100B0939600209277000D
:10156000209278002092790020927A0020927B00CD
:101570002092A50060E070E020926E003CDBB8E0B5
:10158000B093A5007061DBD874FFB0E074FDB1E0EA
:10159000B068B064B7B9B6B1B068B064B6B9B6B146
:1015A000B6FDFDCF04B115B1B6B1BF77B6B9112301
:1015B00009F00FEF0093A600BEDAB8E0B093A500E3
:1015C00070618090B300B2E0B093B300AEDD809262
:1015D000B300F894BFEFB0939200F6DAB0916100D7
:1015E000B0939200B0939300B09394007894B1E0DC
:1015F000B0936100B09363005B2EB0939B00B091F9
:101600009100B0939A007160726020926D0001DDCC
:1016100012DDF7DAF0DA50DB04C087DD2092A50096
:101620007F7E95FF08C0B0B7B860B0BFB5E0B068C6
:10163000B064B7B903C0B0B7B77FB0BFCADB31DCA5
:1016400046DC20D954DC7DDCDCDA32DB35DBA1DBA7
:10165000B0B7B860B0BFB4E0B068B064B7B9B4DBDD
:1016600020DC35DC10D9D1D942DC80DCCADA20DBC1
:1016700023DB8FDB95FF04C0B0B7B77FB0BF07C0D7
:10168000B0B7B860B0BFB5E0B068B064B7B9A1DBBF
:1016900008DC1DDC1CD92BDC88DCB3DA09DB0CDBB5
:1016A00078DB95FF08C0B0B7B860B0BFB5E0B068F0
:1016B000B064B7B903C0B0B7B77FB0BF85DBF1DBAB
:1016C00006DC41D914DC86DC9CDAF2DAF5DA61DB7F
:1016D000B0B7B860B0BFB4E0B068B064B7B979DB98
:1016E000E0DBF5DB62D903DC94DC8BDAE1DAE4DA07
:1016F00050DB95FF04C0B0B7B77FB0BF07C0B0B72D
:10170000B860B0BFB5E0B068B064B7B95DDB74FF76
:10171000B0E074FDB1E0B068B064B7B9B6B1B0681C
:10172000B064B6B9BEDBD3DBE2DB85DC6ADAC0DAF3
:10173000C3DA01DA2EDB71FF25C067FD23C0B0914B
:101740009500B0939200B0939300B0919100B09344
:101750009A00B1E0B0939B0014E624E1B0916D00D3
:10176000B11750F07D7F746020936C00BFEFB09391
:101770009200B093930006C0B0918D00B13008F094
:1017800050CF26C072FF10C067FD0EC0B0916C0034
:10179000BA9511F47B7F41CFB0936C00B0918D006E
:1017A000B13008F03ECF14C0B0919000B23880F450
:1017B000B92FBF7121F4B0916600BB2349F0B091FD
:1017C000740000EF67FF01C000E6B01708F429CFEE
:1017D000F89464DC8090B300B2E0B093B300A5DC71
:1017E0008092B300209261002092620020926300F8
:1017F000522C209296007E7F7894A1D74FDCB92F8F
:10180000BF7129F4B0916600BB2309F481CD48CEA5
:10181000EDE0F0E023D00A3509F01BC0EEE0F0E087
:101820001DD0053A09F015C03AE0ACEAB0E0E3E0BB
:10183000F0E014D00D9331963A95D9F735E1A8EB45
:10184000B0E0EFE0F0E00AD00D9331963A95D9F789
:1018500002C02FDC0AD0E4E2F0E00895E199FECF67
:10186000EEBBFFBBE09A0DB308951ED03AE0ACEAA0
:10187000B0E0E3E0F0E00D910FD031963A95D9F762
:1018800035E1A8EBB0E0EFE0F0E00D9105D0319646
:101890003A95D9F712D00895E199FECF0DBBEEBB72
:1018A000FFBBE29AE19A0895EDE0F0E00FEFF4DF7C
:1018B000EEE0F0E00FEFF0DF0895EDE0F0E00AE594
:1018C000EBDFEEE0F0E005EAE7DF08953091A900F4
:1018D0000091AA00313011F40093B000323011F4BD
:1018E0000093B100333011F40093B200343011F49E
:1018F0000093BE00353011F40093C700363011F468
:101900000093BF00373011F40093B300383011F466
:101910000093C800393011F40093B4003A3011F448
:101920000093B500089525E014D72A95E9F70895A6
:101930001BD71DD71FD721D706D716D718D71AD729
:101940001CD701D711D713D715D717D7089515D797
:1019500011D70DD709D7F7D610D70CD708D704D78A
:10196000F2D60BD707D703D7FFD608958090A900EA
:101970009090AA00F9D6F8D6F7D6E5D68A94D1F792
:10198000FCD6E1D69A94E1F70895F894D1DF7894E3
:10199000CADFC9DFB1E0B093A900B1E0B093AA00FB
:1019A0002092AB00F894E2DF7894B5E06B2E709053
:1019B0008D00CFD6B0918D007B16C9F7B13018F0ED
:1019C000BF3F40F107C082DFF8944FDFB1DFB8E0DE
:1019D000B1BDA9DF6A9459F7B091AB00B395B0934C
:1019E000AB00B33008F4DECF9EDFB091AA00B39510
:1019F000B093AA00F894B091A900BA95E6E4F0E09B
:101A0000EB0FF21D049178940395B091AA00B017E2
:101A100008F4C6CF88DF87DFB091A900B395B093F3
:101A2000A900B091A900BB3008F4B7CF42DBF8940D
:081A30001CDFB8E0B1BD77DF57
:00000001FF
